:10000000080C2500D10C02006607040A6606060AE1
:1000100061006607090A01022E00220C8E00030609
:10002000040A1B0C8E000306180A200CE501040AC2
:10003000080C0600D60C0200580289019C014306F8
:100040007E0AC3047C00690068007E007F007A009D
:10005000BA02300C24006A00A3050509A304430674
:100060002C0A0F0220003F0C84013F0E43063B0A7E
:10007000A402AA022C0A12024306010DFF0FA404D7
:100080003200A40513024306010DFF0FA404330040
:10009000A4051F02A4043600090C24007E0A0802ED
:1000A000E20100080008000800080208030805082B
:1000B00007080A080D08120816081C082208290853
:1000C0003008380841084A0854085F086A0876086A
:1000D000830890089E08AD08BC08CC08DC08ED0831
:1000E000FF08090C2E00400003042F000F032D030E
:1000F0000306CC01EE02750A2C0000080400FF0C78
:100100002D002E002F00090C24000B0C3D007F0059
:1001100047040000AC094706940ACA096606C705E9
:1001200067066B06940A4605FC0C3F024306A40AC8
:10013000DF01FD02A00A0306130BBD020000870ABF
:10014000DF020306F20B870A0000A60AC706BF02F9
:10015000C704FE03880A290A66070008BF027E005A
:100160004705CA0966070008BF0200001C02890192
:1001700038007802A706C50A4F0929000304E706DC
:1001800029034704DF03AC0A290A0000C70AC80A8A
:10019000C90AC10AC103DC0A09029C004306F70A26
:1001A0000306D50ABC021202D80AFC001302870516
:1001B0002100000000000008FA02E80A06052605F2
:1001C0001C0200000000000000000000E70A000818
:1001D0001A029C000706F20A000003060604030741
:1001E0000605000803062604030726050008870401
:1001F00009026706F502010B3500D60667044604BE
:1002000000086707F50300080B02670E100D3500A4
:10021000D60667050008100C8400070E4306F10B94
:10022000C706BF02170B090C3D00A4027F0047045C
:10023000C704AC094706230BCA096606C70567064B
:100240006106230B4604FC0C3F0243060B0BDF0147
:10025000FD026E0B0306130B79000A028B018C0161
:100260008D018E018F014307E40B6A026B026C0261
:100270006D026E02CA09E400080C0600A4050A0219
:10028000EA075C0B98014307550B0B0299014307E2
:10029000550B2C0C2400B407550B2706550BA30552
:1002A0004F0A540B27067E0A680B0A02F00E700FE5
:1002B00043077E0AA305EE0A4306510BB4079001DB
:1002C0004306520B1A027F0E2704430727058A01B3
:1002D0004307550B2B0C2400A3054F0A00006003B5
:1002E000DF02160BF40B3E0243067F0B9E00800BD1
:1002F00011023D023F0743060706E706730B96000F
:100300002C002A0003042C038A030F0EEC012F009B
:100310000F03EC01AC02040C88002D0071092C03C2
:100320002D032C032D032C032D032C032D030C066E
:100330009C0B1102CD010306FF0C2900A404CA097D
:10034000A4056B0017024306D70B7F0E2C000A0290
:100350002D0071090C022A00F707B10B040C88006C
:10036000B30B48021F0E2E008E076E06C20B2F0025
:100370004306BF0B03042A032B03EE02BB0B0A0246
:100380008C00D70B03040A03CA012C00070C8E0053
:100390002D0003040D03EC010D06AC0271096D0381
:1003A0006C036D036C036D036C038C028A00F7070A
:1003B000DF0BC90103072900A705A4047E0A8900F1
:1003C00003062900DC0B0000E50BE60BCA09E80B6D
:1003D000E90BEA0BEB0B00007E0AEE0BEF0BF00BC8
:0E03E00000000000B902F907F60B000AE30B5B
:10040000840C2700310A800C060A830C2700A00CFC
:10041000C6042900080C2800E6046903C604030684
:10042000C6050000E605E8020C0A0000E60400002C
:10043000C60500000000E605C606E704E604E70777
:10044000470A07020F0EE2012B0A2E0A470A2B0A5F
:10045000310A360A470AA7020A02090AA7020F024E
:10046000090AE605C605A702A10C080AC605000090
:10047000E605080C2800E6050305C60703046F031C
:10048000E604C605E8023B0AE6050000E604C604E9
:10049000E6054A0A4B0AC605E7070008010880037B
:1004A0002F000F03070EE201870AD80B910B9E0B5A
:1004B0005D0B550BF90B0B02F90F4306170B0002EE
:1004C0002A00A40200022B00A40200022C00F30A5E
:1004D0002400070C4C017E098C07750A6C0620016C
:1004E000FF0F6C0760010402000B400143067B0A0A
:1004F0006C06280BF90B6C07280BF90BE2010108BD
:10050000020804080808100820084008800880062F
:10051000CB0B0003070EE201BF0BF90BF90BF90B34
:10052000F90BF90BF90BF90B5F07990AFF06A00A03
:10053000B00A7F079E0A8706A00AB00A8007B00AA1
:100540000706A90A5406AB0A1F0786053F07A6043B
:1005500000085406A40A1F0786043F07A6050008E2
:100560001F0786043F07A604000847046704000F1E
:1005700043063008010F43063108030F43063208D3
:10058000010F43063308070F43063608010F4306E1
:100590003708150F43063808010F43063908030FC3
:1005A00043063A080E0F430634082C0F43063B0857
:1005B000010F43063C08030F43063D08040F4306A2
:1005C0003E08090F43063F086705390F4306070831
:1005D000010F43060D0867044705FF0804020F0ECC
:1005E0000C0F43073D0B0B02B5094706F90B6706D5
:1005F0006A07FC0A3500350C4A07680A6A071C0BB3
:100600000F0E2A000509670000028F014306A304AC
:100610004306290A00022F00D406100BD405FB0B59
:1006200003094306100B6700A304D404000A0A025E
:100630002000400075001F0B67063B0B0F0E2A00C1
:100640000509670000028F014307A30443077E0AE0
:10065000C3062C0BC305FB0B310C2600090C2E0026
:100660006F000400EF03320BEE02300B6600C30490
:10067000A404A3047E0A8001240B0A027D0FF70E56
:1006800043064E0B010F4306520B0A02070ED5011B
:10069000B5094706F90B6A071C0B000BEB000304B6
:1006A0006B036B030A02070E4B0B8007F90B8003E9
:1006B000F00EA4043B010F0F650B9409800634056E
:1006C00000020F0EA4043B01F00F5B013B002F0062
:1006D000A4055B014306700BBF0667054605750B55
:1006E000DF06750BBF06670446040F025C01430674
:1006F000810BFF055F06840B1F067F0BA605860591
:10070000840B1F068604FF040F025D0143068D0B58
:100710003F06A6053F07E705F90B3F06A604E704D9
:10072000F90B1406A00BFA06A20B0707AB0BA404E7
:100730001C024306070469006800F90B1406930BBA
:10074000FA06950B0706AB0BA4041C02430607052B
:1007500069006800F90BA70440031E0E28008006FC
:100760000805340708043407940908024306C80B37
:10077000FD0E4306C20B9406F90BA304780B080C7C
:100780000600660006042604A4047A00BA027C006F
:1007900069006800F90B0C023A000002120F4306D0
:1007A000FA04010F4306FA053A0C24001A02000B62
:1007B00000023F0F4307F90BA402E006E60B140604
:1007C000E80BFA06EA0B0706970BEC0B1406E10B95
:1007D000FA06E30B0707A40B00032F000F031F0EFD
:1007E000280040039F07290034059F06B50BA70585
:0C07F000F90BD404C304A304A4047E0A83
:0207FE00700C7D
:021FFE00EE0FE4
:00000001FF
